:0400000000000000FC
:0400010000000000FB
:0400020000000000FA
:0400030000000000F9
:0400040000000000F8
:0400050000000000F7
:0400060000000000F6
:0400070000000000F5
:0400080000000000F4
:0400090000000000F3
:04000A0000000000F2
:04000B0000000000F1
:04000C0000000000F0
:04000D000FC6C0005A
:04000E0016200201B5
:04000F002EC60000F9
:040010003520020095
:0400110000000000EB
:0400120000000000EA
:0400130000000000E9
:0400140000000000E8
:0400150008B237E115
:04001600098A16211C
:0400170000000000E5
:04001800320402C1EB
:0400190000000000E3
:04001A0000000000E2
:04001B0000000000E1
:04001C0000000000E0
:04001D0000000000DF
:04001E0000000000DE
:04001F002150000F5D
:040020002AC6000EDE
:0400210027C601C12C
:04002200109017E93A
:0400230019E60024B6
:0400240033E60004BB
:04002500180404B700
:04002600343C400026
:04002700098A16210B
:040028001504046156
:0400290039E6182577
:04002A0039E6182576
:04002B00320405771F
:04002C00063C50003E
:04002D002FE6404535
:04002E00340405D7BA
:04002F00063C50003B
:040030003E04060F75
:0400310000000000CB
:00000001ff
